:10000000A20119299000A31727308F001030142067
:1000100003308F00E83014208F01643014208F01EA
:100020000A30142010081F288E0011088D001008B7
:100030008C00E2200C08031DA313A31B0800303E14
:10004000A2184828930005108316051083123A3031
:100050008D009830A82085108316851083123330C8
:10006000920083160F308605831223175420231322
:100070005420223092005420283047200C30472052
:100080000630472001304720A214130848282214C4
:100090009200231785102218532823138514221445
:1000A000FE3C03191429221C22100F308605120869
:1000B000F039860405140510920E221854281330C6
:1000C000231F03018D007830A82003141429A400F5
:1000D00082200A309A2024088004841380068C0130
:1000E0008D018417240880066400800684130005AF
:1000F0000319802810088C0703188D0F71288D03B1
:100100000D08142980048428FF3A841780051429D7
:10011000890083160814831208081429880083169E
:10012000081555308900AA30890088148818962847
:10013000081114298F018E00FF308E07031C8F07D2
:10014000031C142903308D00DF30A8209C288D016A
:10015000E83E8C008D09FC30031CB1288C07031885
:10016000AE288C0764008D0FAE280C18B7288C1CA5
:10017000BB280000BB2808008D018F018E000230D3
:10018000CB288D018F018E000130CB288D018F018E
:100190008E000430CB2894000F080D02031DD228D6
:1001A0000E080C0204300318013003190230140544
:1001B000031DFF3014290038031DFF300405031D03
:1001C000FF30142910309200910190010D0D900D17
:1001D000910D0E0890020F08031C0F0F91020318D7
:1001E000F8280E0890070F0803180F0F9107031047
:1001F0008C0D8D0D920BE6280C08142910309400FC
:100200008D018C01930C920C031C0C290E088C0799
:100210000F0803180F0F8D078D0C8C0C910C900C90
:10022000940B02291008142983130313831264000A
:10023000080010308500373062001030BC000230FA
:10024000B9000230BB0001308820B70037088C00AD
:100250003730BC209E0064001E0803193629023086
:100260008820B20003308820B3003A292830B20039
:100270002330B300FE3020200130202046302020E3
:100280003830202042302020593020204330202098
:100290002030202054302020453020204C30202099
:1002A0004530202056302020493020205330202057
:1002B000493020204F3020204E302020FF30900049
:1002C0000630840002306720BA00B4013A088C007E
:1002D0000530C1209E003A088C001030C620A000D6
:1002E0001E0884002008DB20A000A1006400200874
:1002F000210403197D290130B4003A088C00103024
:10030000C1209E003A088C001930C620A0001E08AB
:1003100084002008DB20A000A10064002008210444
:10032000031994290230B4003A088C001930C12016
:100330009E003A088C003230C620A0001E088400BF
:100340002008DB20A000A10064002008210403197C
:10035000AB290330B40034088C000330BC209E006D
:1003600064001E080319C429B90A01308F002C301B
:100370009B2039088C000730BC209E0064001E08BA
:100380000319C4290330B90039088C000330BC209C
:100390009E0064001E0803193A2A36089200930151
:1003A0008E0101308F00FE209E0011089F0038084A
:1003B0001E07A8001F080318013EA90028088C008A
:1003C00029088D000A308E008F01E220AC000D0854
:1003D000AD0028088C0029088D000A308E008F019E
:1003E000E2201008AE001108AF002C0892002D0882
:1003F000930004308E008F01FE20AC001108AD0088
:100400002E0892002F08930004308E008F01FE20EA
:10041000AE001108AF002E088C002F088D000A30A6
:100420008E008F01E220AE000D08AF002C082E07D1
:10043000A8002D080318013E2F07A900FE30202038
:1004400001302020493020204E3020203A3020201A
:100450002030202020302020290891002808022068
:10046000203020204B302020483020207A3020209F
:100470002030202039088C000430BC209E0064000D
:100480001E080319822A34088C000130BC209E000B
:1004900064001E0803194F2AB20A0319B30A34086C
:1004A0008C000230BC209E0064001E0803195E2AE6
:1004B0000130B2020030031C013EB3020230890059
:1004C00032088E200330890033088E2001308900E5
:1004D00037308E20FE302020013020204F30202069
:1004E0004C3020203A30202033089100320802207E
:1004F000203020204D302020683020207A302020ED
:100500002030202039088C000530BC209E0064007B
:100510001E080319B52A32082C07B0003308031847
:10052000013E2D07B100FE30202001302020313067
:10053000202030302020473020203A30202020302A
:10054000202031089100300802202E3020202F0872
:1005500091002E080220203020204D3020206830CD
:1005600020207A302020203020205223360892008C
:1005700093018E0101308F00FE209E0011089F0024
:1005800038081E07A8001F080318013EA900280804
:100590008C0029088D007D308E008F01E220AC0098
:1005A0000D08AD0028088C0029088D007D308E00D4
:1005B0008F01E2201008AE001108AF002C08920055
:1005C0002D08930040308E008F01FE20AC001108F2
:1005D000AD002E0892002F08930040308E008F014E
:1005E000FE20AE001108AF002E088C002F088D00F1
:1005F0007D308E008F01E220AE000D08AF002C0888
:100600002E07A8002D080318013E2F07A900BB30B4
:10061000A8021230031C013EA90228088C002908F8
:100620008D000A308E008F01E220AC000D08AD0075
:100630002C0892002D0893000A308E008F01FE20B6
:100640009E0011089F001E082802AE001F08031C10
:10065000013E2902AF00FE302020C0302020423071
:10066000202049302020533020203A3020202030D4
:100670002020203020202D0891002C0802202E3030
:1006800020202F0891002E080220203020204D30FD
:100690002020683020207A30202020302020643034
:1006A0009A205E298101BC153C0865003B08B50015
:1006B0000000B50B582B0000000073237323732335
:1006C00073237323BC113C0865000108B600B50113
:1006D000B50A85158511010836020319682BB5097D
:1006E000350AB8007D2B6130B5000000772B782BE0
:0C06F000792B7A2BB50B792B0800080041
:084000007F007F007F007F00BC
:04400E00F53F010079
:00000001FF
